LX51 LINKER/LOCATER V4.06                                                               05/20/2006  16:12:40  PAGE 1


LX51 LINKER/LOCATER V4.06, INVOKED BY:
C:\KEIL\C51\BIN\LX51.EXE COMMON {C_root.obj}, BANK0 {C_bank0.obj}, BANK1 {C_bank1.obj}, BANK2 {C_bank2.obj}, COMMON {L51
>> IBank.obj} TO L51IBANK BANKAREA (0X000000, 0X00FFFF) CLASSES (HDATA (X:0X10000-X:0X7FFFF))


CPU MODE:     8051 MODE
MEMORY MODEL: SMALL


INPUT MODULES INCLUDED:
  C_root.obj (C_ROOT)
         COMMENT TYPE 0: C51 V8.04
  C_bank0.obj (C_BANK0)
         COMMENT TYPE 0: C51 V8.04
  C_bank1.obj (C_BANK1)
         COMMENT TYPE 0: C51 V8.04
  C_bank2.obj (C_BANK2)
         COMMENT TYPE 0: C51 V8.04
  L51IBank.obj (?BANK?SWITCHING)
         COMMENT TYPE 0: AX51 V3.01
  C:\KEIL\C51\LIB\C51NS.LIB (?C?ISTPTR)
         COMMENT TYPE 1: A51 / ASM51 Assembler
  C:\KEIL\C51\LIB\C51NS.LIB (PRINTF)
         COMMENT TYPE 1: A51 / ASM51 Assembler
  C:\KEIL\C51\LIB\C51NS.LIB (?C?STRCPY517)
         COMMENT TYPE 1: A51 / ASM51 Assembler
  C:\KEIL\C51\LIB\C51NS.LIB (?C?CLDPTR)
         COMMENT TYPE 1: A51 / ASM51 Assembler
  C:\KEIL\C51\LIB\C51NS.LIB (?C?CSTPTR)
         COMMENT TYPE 1: A51 / ASM51 Assembler
  C:\KEIL\C51\LIB\C51NS.LIB (?C?PLDIIDATA)
         COMMENT TYPE 1: A51 / ASM51 Assembler
  C:\KEIL\C51\LIB\C51NS.LIB (?C?CCASE)
         COMMENT TYPE 1: A51 / ASM51 Assembler
  C:\KEIL\C51\LIB\C51NS.LIB (PUTCHAR)
         COMMENT TYPE 1: A51 / ASM51 Assembler


ACTIVE MEMORY CLASSES OF MODULE:  L51IBANK (C_ROOT)

BASE        START       END         USED      MEMORY CLASS
==========================================================
X:000000H   X:010000H   X:07FFFFH   0000C8H   HDATA
C:000000H   C:000000H   C:00FFFFH   0007FAH   CODE
I:000000H   I:000000H   I:00007FH   000022H   DATA
X:000000H   X:000000H   X:00FFFFH   00012CH   XDATA
I:000000H   I:000000H   I:0000FFH   000001H   IDATA
I:000020H.0 I:000020H.0 I:00002FH.7 000001H.1 BIT


MEMORY MAP OF MODULE:  L51IBANK (C_ROOT)


START     STOP      LENGTH    ALIGN  RELOC    MEMORY CLASS   SEGMENT NAME
=========================================================================

* * * * * * * * * * *   D A T A   M E M O R Y   * * * * * * * * * * * * *
000000H   000007H   000008H   ---    AT..     DATA           "REG BANK 0"
000008H   00001DH   000016H   BYTE   UNIT     DATA           _DATA_GROUP_
00001EH.0 00001FH.7 000002H.0 ---    ---      **GAP**
000020H.0 000021H.0 000001H.1 BIT    UNIT     BIT            _BIT_GROUP_
000021H.1 000021H   000000H.7 ---    ---      **GAP**
000022H   000025H   000004H   BYTE   UNIT     DATA           ?DT?C_BANK0
000026H   000026H   000001H   BYTE   UNIT     IDATA          ?STACK

* * * * * * * * * * *   C O D E   M E M O R Y   * * * * * * * * * * * * *
LX51 LINKER/LOCATER V4.06                                                             05/20/2006  16:12:40  PAGE 2



***   CODE BANK 0   ***
000006H   000006H   000001H   BYTE   UNIT     CODE/B0        ?PR?INTRP0?C_BANK0
000007H   00000DH   000007H   ---    ---      **GAP**
00000EH   000019H   00000CH   BYTE   UNIT     CODE/B0        ?PR?FUNC0?C_BANK0

***   CODE BANK 1   ***
000006H   000006H   000001H   BYTE   UNIT     CODE/B1        ?PR?INTRP1?C_BANK1
000007H   00000DH   000007H   ---    ---      **GAP**
00000EH   000019H   00000CH   BYTE   UNIT     CODE/B1        ?PR?FUNC1?C_BANK1

***   CODE BANK 2   ***
00000EH   000016H   000009H   BYTE   UNIT     CODE/B2        ?PR?FUNC2?C_BANK2

***   CODE BANK 3   ***
00000EH   00007FH   000072H   BYTE   UNIT     CODE/B3        ?CO?C_ROOT
000080H   0000AFH   000030H   BYTE   UNIT     CODE/B3        ?CO?C_BANK0
0000B0H   0000DFH   000030H   BYTE   UNIT     CODE/B3        ?CO?C_BANK1
0000E0H   0000FFH   000020H   BYTE   UNIT     CODE/B3        ?CO?C_BANK2

***   COMMON AREA   ***
000000H   000002H   000003H   ---    OFFS..   CODE           ?CO?L51IBANK?3
000003H   000005H   000003H   BYTE   OFFS..   CODE           ?C_BANK0?00003
000006H   00000AH   000005H   ---    ---      **GAP**
00000BH   00000DH   000003H   BYTE   OFFS..   CODE           ?C_BANK1?0000B
00000EH   0000FFH   0000F2H   ---    ---      **GAP**
000100H   000480H   000381H   BYTE   UNIT     CODE           ?PR?PRINTF?PRINTF
000481H   000709H   000289H   BYTE   UNIT     CODE           ?C?LIB_CODE
00070AH   00078DH   000084H   BYTE   UNIT     CODE           ?PR?MAIN?C_ROOT
00078EH   0007B4H   000027H   BYTE   UNIT     CODE           ?PR?PUTCHAR?PUTCHAR
0007B5H   0007C9H   000015H   BYTE   UNIT     CODE           ?C_C51STARTUP
0007CAH   0007DBH   000012H   BYTE   UNIT     CODE           ?BANK?SELECT

* * * * * * * * * * *  X D A T A   M E M O R Y  * * * * * * * * * * * * *
000000H   00012BH   00012CH   BYTE   UNIT     XDATA          ?XD?C_ROOT
00012CH   00FFFFH   00FED4H   ---    ---      **GAP**
010000H   0100C7H   0000C8H   BYTE   INSEG    HDATA          ?FD?C_ROOT



OVERLAY MAP OF MODULE:   L51IBANK (C_ROOT)


FUNCTION/MODULE              BIT_GROUP   DATA_GROUP 
--> CALLED FUNCTION/MODULE  START  STOP  START  STOP
====================================================
INTRP0/C_BANK0              ----- -----  ----- -----

*** NEW ROOT **************

INTRP1/C_BANK1              ----- -----  ----- -----

*** NEW ROOT **************

?C_C51STARTUP               ----- -----  ----- -----
  +--> ?PR?MAIN?C_ROOT

MAIN/C_ROOT                 ----- -----  0008H 0009H
  +--> ?CO?C_ROOT
  +--> ?PR?PRINTF?PRINTF
  +--> ?PR?FUNC0?C_BANK0
  +--> ?PR?FUNC1?C_BANK1

?CO?C_ROOT                  ----- -----  ----- -----

LX51 LINKER/LOCATER V4.06                                                             05/20/2006  16:12:40  PAGE 3


PRINTF/PRINTF               20H.0 21H.0  000AH 001DH
  +--> ?PR?PUTCHAR?PUTCHAR

PUTCHAR/PUTCHAR             ----- -----  ----- -----

FUNC0/C_BANK0               ----- -----  ----- -----
  +--> ?CO?C_BANK0
  +--> ?PR?PRINTF?PRINTF
  +--> ?PR?FUNC2?C_BANK2

?CO?C_BANK0                 ----- -----  ----- -----

FUNC2/C_BANK2               ----- -----  ----- -----
  +--> ?CO?C_BANK2
  +--> ?PR?PRINTF?PRINTF

?CO?C_BANK2                 ----- -----  ----- -----

FUNC1/C_BANK1               ----- -----  ----- -----
  +--> ?CO?C_BANK1
  +--> ?PR?PRINTF?PRINTF
  +--> ?PR?FUNC2?C_BANK2

?CO?C_BANK1                 ----- -----  ----- -----



INTERBANK CALL TABLE OF MODULE:  L51IBANK (C_ROOT)

ADDRESS     FUNCTION NAME
-------------------------
C:0007CAH   func1
C:0007D0H   intrp1
C:0007D6H   func2



PUBLIC SYMBOLS OF MODULE:  L51IBANK (C_ROOT)


      VALUE       CLASS    TYPE      PUBLIC SYMBOL NAME
      =================================================
      0000000AH   DATA     ---       ?_PRINTF517?BYTE
      0000000AH   DATA     ---       ?_PRINTF?BYTE
      0000000AH   DATA     ---       ?_SPRINTF517?BYTE
      0000000AH   DATA     ---       ?_SPRINTF?BYTE
      00000003H   NUMBER   ---       ?B_CB
      00000094H   DATA     ---       ?B_CURRENTBANK
      00000004H   NUMBER   ---       ?B_FACTOR
      00000000H   NUMBER   ---       ?B_IB
      00000094H   DATA     ---       ?B_MEX1
      00000008H   NUMBER   ---       ?B_MODE
      00000004H   NUMBER   ---       ?B_NBANKS
      00000000H   NUMBER   ---       ?B_RST_BANK
      010006E4H   CODE     ---       ?C?CCASE
      0100069FH   CODE     ---       ?C?CLDPTR
      01000481H   CODE     NEAR LAB  ?C?CLDXPTR
      00000000H   NUMBER   ---       ?C?CODESEG
      010006BDH   CODE     ---       ?C?CSTPTR
      01000499H   CODE     NEAR LAB  ?C?CSTXPTR
      00000093H   DATA     BYTE      ?C?DPSEL
      010004B1H   CODE     NEAR LAB  ?C?ILDXPTR
      0100056DH   CODE     ---       ?C?ISTPTR
      010004CDH   CODE     NEAR LAB  ?C?ISTXPTR
      01000529H   CODE     NEAR LAB  ?C?LLDXPTR
LX51 LINKER/LOCATER V4.06                                                             05/20/2006  16:12:40  PAGE 4


      0100054BH   CODE     NEAR LAB  ?C?LSTXPTR
      010006D4H   CODE     ---       ?C?PLDIIDATA
      010004E9H   CODE     NEAR LAB  ?C?PLDXPTR
      01000508H   CODE     NEAR LAB  ?C?PSTXPTR
      01000659H   CODE     ---       ?C?STRCPY517
      00000000H   NUMBER   ---       ?C?XDATASEG
      00000008H   NUMBER   ---       ?C?XPAGE1RST
      00000096H   DATA     ---       ?C?XPAGE1SFR
      0100070AH   CODE     ---       ?C_START
      01000000H   CODE     NEAR LAB  ?C_STARTUP
      01000162H   CODE     ---       _PRINTF
      01000162H   CODE     ---       _PRINTF517
      0100078EH   CODE     ---       _PUTCHAR
      0100015CH   CODE     ---       _SPRINTF
      0100015CH   CODE     ---       _SPRINTF517
*SFR* 000000D0H.6 DATA     BIT       AC
*SFR* 000000E0H   DATA     BYTE      ACC
*SFR* 000000F0H   DATA     BYTE      B
*SFR* 000000D0H.7 DATA     BIT       CY
*SFR* 00000083H   DATA     BYTE      DPH
*SFR* 00000082H   DATA     BYTE      DPL
*SFR* 000000A8H.7 DATA     BIT       EA
*SFR* 000000A8H.4 DATA     BIT       ES
*SFR* 000000A8H.1 DATA     BIT       ET0
*SFR* 000000A8H.3 DATA     BIT       ET1
*SFR* 000000A8H   DATA     BIT       EX0
*SFR* 000000A8H.2 DATA     BIT       EX1
*SFR* 000000D0H.5 DATA     BIT       F0
      02010000H   HDATA    ---       farr
      0080000EH   CODE/B0  ---       func0
      0081000EH   CODE/B1  ---       func1
      0082000EH   CODE/B2  ---       func2
*SFR* 000000A8H   DATA     BYTE      IE
*SFR* 00000088H.1 DATA     BIT       IE0
*SFR* 00000088H.3 DATA     BIT       IE1
*SFR* 000000B0H.2 DATA     BIT       INT0
*SFR* 000000B0H.3 DATA     BIT       INT1
      00800006H   CODE/B0  ---       intrp0
      00810006H   CODE/B1  ---       intrp1
*SFR* 000000B8H   DATA     BYTE      IP
*SFR* 00000088H   DATA     BIT       IT0
*SFR* 00000088H.2 DATA     BIT       IT1
      0100070AH   CODE     ---       main
*SFR* 00000094H   DATA     BYTE      MEX1
*SFR* 00000095H   DATA     BYTE      MEX2
*SFR* 00000096H   DATA     BYTE      MEX3
*SFR* 00000097H   DATA     BYTE      MEXSP
*SFR* 000000D0H.2 DATA     BIT       OV
*SFR* 000000D0H   DATA     BIT       P
*SFR* 00000080H   DATA     BYTE      P0
*SFR* 00000090H   DATA     BYTE      P1
*SFR* 000000A0H   DATA     BYTE      P2
*SFR* 000000B0H   DATA     BYTE      P3
*SFR* 00000087H   DATA     BYTE      PCON
*SFR* 000000A0H   DATA     BYTE      PPAGE_SFR
*SFR* 000000B8H.4 DATA     BIT       PS
*SFR* 000000D0H   DATA     BYTE      PSW
*SFR* 000000B8H.1 DATA     BIT       PT0
*SFR* 000000B8H.3 DATA     BIT       PT1
*SFR* 000000B8H   DATA     BIT       PX0
*SFR* 000000B8H.2 DATA     BIT       PX1
*SFR* 00000098H.2 DATA     BIT       RB8
*SFR* 000000B0H.7 DATA     BIT       RD
*SFR* 00000098H.4 DATA     BIT       REN
*SFR* 00000098H   DATA     BIT       RI
LX51 LINKER/LOCATER V4.06                                                             05/20/2006  16:12:40  PAGE 5


*SFR* 000000D0H.3 DATA     BIT       RS0
*SFR* 000000D0H.4 DATA     BIT       RS1
*SFR* 000000B0H   DATA     BIT       RXD
*SFR* 00000099H   DATA     BYTE      SBUF
*SFR* 00000098H   DATA     BYTE      SCON
*SFR* 00000098H.7 DATA     BIT       SM0
*SFR* 00000098H.6 DATA     BIT       SM1
*SFR* 00000098H.5 DATA     BIT       SM2
*SFR* 00000081H   DATA     BYTE      SP
*SFR* 000000B0H.4 DATA     BIT       T0
*SFR* 000000B0H.5 DATA     BIT       T1
*SFR* 00000098H.3 DATA     BIT       TB8
*SFR* 00000088H   DATA     BYTE      TCON
*SFR* 00000088H.5 DATA     BIT       TF0
*SFR* 00000088H.7 DATA     BIT       TF1
*SFR* 0000008CH   DATA     BYTE      TH0
*SFR* 0000008DH   DATA     BYTE      TH1
*SFR* 00000098H.1 DATA     BIT       TI
*SFR* 0000008AH   DATA     BYTE      TL0
*SFR* 0000008BH   DATA     BYTE      TL1
*SFR* 00000089H   DATA     BYTE      TMOD
*SFR* 00000088H.4 DATA     BIT       TR0
*SFR* 00000088H.6 DATA     BIT       TR1
*SFR* 000000B0H.1 DATA     BIT       TXD
      00000022H   DATA     DWORD     ul
*SFR* 000000B0H.6 DATA     BIT       WR
      02000000H   XDATA    ---       xarr
      020000C8H   XDATA    ---       xstr



SYMBOL TABLE OF MODULE:  L51IBANK (C_ROOT)

      VALUE       REP       CLASS    TYPE      SYMBOL NAME
      ====================================================
      ---         MODULE    ---      ---       C_ROOT
      020000C8H   PUBLIC    XDATA    ---       xstr
      02000000H   PUBLIC    XDATA    ---       xarr
      02010000H   PUBLIC    HDATA    ---       farr
      0100070AH   PUBLIC    CODE     ---       main
      00000080H   SFRSYM    DATA     BYTE      P0
      00000090H   SFRSYM    DATA     BYTE      P1
      000000A0H   SFRSYM    DATA     BYTE      P2
      000000B0H   SFRSYM    DATA     BYTE      P3
      000000B0H.4 SFRSYM    DATA     BIT       T0
      000000D0H.6 SFRSYM    DATA     BIT       AC
      000000B0H.5 SFRSYM    DATA     BIT       T1
      000000A8H.7 SFRSYM    DATA     BIT       EA
      000000A8H   SFRSYM    DATA     BYTE      IE
      000000B0H.7 SFRSYM    DATA     BIT       RD
      000000A8H.4 SFRSYM    DATA     BIT       ES
      000000B8H   SFRSYM    DATA     BYTE      IP
      00000098H   SFRSYM    DATA     BIT       RI
      000000B0H.2 SFRSYM    DATA     BIT       INT0
      000000D0H.7 SFRSYM    DATA     BIT       CY
      00000098H.1 SFRSYM    DATA     BIT       TI
      000000B0H.3 SFRSYM    DATA     BIT       INT1
      000000B8H.4 SFRSYM    DATA     BIT       PS
      00000081H   SFRSYM    DATA     BYTE      SP
      000000D0H.2 SFRSYM    DATA     BIT       OV
      000000B0H.6 SFRSYM    DATA     BIT       WR
      00000099H   SFRSYM    DATA     BYTE      SBUF
      00000087H   SFRSYM    DATA     BYTE      PCON
      00000098H   SFRSYM    DATA     BYTE      SCON
      00000089H   SFRSYM    DATA     BYTE      TMOD
LX51 LINKER/LOCATER V4.06                                                             05/20/2006  16:12:40  PAGE 6


      00000088H   SFRSYM    DATA     BYTE      TCON
      00000088H.1 SFRSYM    DATA     BIT       IE0
      00000088H.3 SFRSYM    DATA     BIT       IE1
      000000F0H   SFRSYM    DATA     BYTE      B
      000000E0H   SFRSYM    DATA     BYTE      ACC
      000000A8H.1 SFRSYM    DATA     BIT       ET0
      000000A8H.3 SFRSYM    DATA     BIT       ET1
      00000088H.5 SFRSYM    DATA     BIT       TF0
      00000088H.7 SFRSYM    DATA     BIT       TF1
      00000098H.2 SFRSYM    DATA     BIT       RB8
      0000008CH   SFRSYM    DATA     BYTE      TH0
      000000A8H   SFRSYM    DATA     BIT       EX0
      00000088H   SFRSYM    DATA     BIT       IT0
      0000008DH   SFRSYM    DATA     BYTE      TH1
      00000098H.3 SFRSYM    DATA     BIT       TB8
      000000A8H.2 SFRSYM    DATA     BIT       EX1
      00000088H.2 SFRSYM    DATA     BIT       IT1
      000000D0H   SFRSYM    DATA     BIT       P
      00000098H.7 SFRSYM    DATA     BIT       SM0
      0000008AH   SFRSYM    DATA     BYTE      TL0
      00000098H.6 SFRSYM    DATA     BIT       SM1
      0000008BH   SFRSYM    DATA     BYTE      TL1
      00000098H.5 SFRSYM    DATA     BIT       SM2
      000000B8H.1 SFRSYM    DATA     BIT       PT0
      000000B8H.3 SFRSYM    DATA     BIT       PT1
      000000D0H.3 SFRSYM    DATA     BIT       RS0
      00000088H.4 SFRSYM    DATA     BIT       TR0
      000000D0H.4 SFRSYM    DATA     BIT       RS1
      00000088H.6 SFRSYM    DATA     BIT       TR1
      000000B8H   SFRSYM    DATA     BIT       PX0
      000000B8H.2 SFRSYM    DATA     BIT       PX1
      00000083H   SFRSYM    DATA     BYTE      DPH
      00000082H   SFRSYM    DATA     BYTE      DPL
      00000098H.4 SFRSYM    DATA     BIT       REN
      000000B0H   SFRSYM    DATA     BIT       RXD
      000000B0H.1 SFRSYM    DATA     BIT       TXD
      000000D0H.5 SFRSYM    DATA     BIT       F0
      000000D0H   SFRSYM    DATA     BYTE      PSW

      0100070AH   BLOCK     CODE     ---       LVL=0
      0100070AH   BLOCK     CODE     NEAR LAB  LVL=1
      00000008H   SYMBOL    DATA     WORD      i
      ---         BLOCKEND  ---      ---       LVL=1
      0100070AH   LINE      CODE     ---       #19
      0100070AH   LINE      CODE     ---       #24
      0100070DH   LINE      CODE     ---       #25
      01000710H   LINE      CODE     ---       #26
      01000713H   LINE      CODE     ---       #27
      01000716H   LINE      CODE     ---       #29
      01000725H   LINE      CODE     ---       #31
      0100072AH   LINE      CODE     ---       #32
      01000748H   LINE      CODE     ---       #33
      01000766H   LINE      CODE     ---       #34
      01000774H   LINE      CODE     ---       #36
      0100077DH   LINE      CODE     ---       #37
      01000780H   LINE      CODE     ---       #38
      01000789H   LINE      CODE     ---       #39
      0100078CH   LINE      CODE     ---       #41
      ---         BLOCKEND  ---      ---       LVL=0

      ---         MODULE    ---      ---       C_BANK0
      00000022H   PUBLIC    DATA     DWORD     ul
      00800006H   PUBLIC    CODE/B0  ---       intrp0
      0080000EH   PUBLIC    CODE/B0  ---       func0

LX51 LINKER/LOCATER V4.06                                                             05/20/2006  16:12:40  PAGE 7


      0080000EH   BLOCK     CODE/B0  ---       LVL=0
      0080000EH   LINE      CODE/B0  ---       #13
      0080000EH   LINE      CODE/B0  ---       #14
      00800017H   LINE      CODE/B0  ---       #15
      ---         BLOCKEND  ---      ---       LVL=0

      00800006H   BLOCK     CODE/B0  ---       LVL=0
      00800006H   LINE      CODE/B0  ---       #18
      00800006H   LINE      CODE/B0  ---       #20
      ---         BLOCKEND  ---      ---       LVL=0

      ---         MODULE    ---      ---       C_BANK1
      00810006H   PUBLIC    CODE/B1  ---       intrp1
      0081000EH   PUBLIC    CODE/B1  ---       func1

      0081000EH   BLOCK     CODE/B1  ---       LVL=0
      0081000EH   LINE      CODE/B1  ---       #11
      0081000EH   LINE      CODE/B1  ---       #12
      00810017H   LINE      CODE/B1  ---       #13
      ---         BLOCKEND  ---      ---       LVL=0

      00810006H   BLOCK     CODE/B1  ---       LVL=0
      00810006H   LINE      CODE/B1  ---       #16
      00810006H   LINE      CODE/B1  ---       #18
      ---         BLOCKEND  ---      ---       LVL=0

      ---         MODULE    ---      ---       C_BANK2
      0082000EH   PUBLIC    CODE/B2  ---       func2

      0082000EH   BLOCK     CODE/B2  ---       LVL=0
      0082000EH   LINE      CODE/B2  ---       #9
      0082000EH   LINE      CODE/B2  ---       #10
      ---         BLOCKEND  ---      ---       LVL=0

      ---         MODULE    ---      ---       ?BANK?SWITCHING
      00000003H   PUBLIC    NUMBER   ---       ?B_CB
      00000094H   PUBLIC    DATA     ---       ?B_CURRENTBANK
      00000004H   PUBLIC    NUMBER   ---       ?B_FACTOR
      00000000H   PUBLIC    NUMBER   ---       ?B_IB
      00000094H   PUBLIC    DATA     ---       ?B_MEX1
      00000008H   PUBLIC    NUMBER   ---       ?B_MODE
      00000004H   PUBLIC    NUMBER   ---       ?B_NBANKS
      00000000H   PUBLIC    NUMBER   ---       ?B_RST_BANK
      01000481H   PUBLIC    CODE     NEAR LAB  ?C?CLDXPTR
      01000499H   PUBLIC    CODE     NEAR LAB  ?C?CSTXPTR
      00000093H   PUBLIC    DATA     BYTE      ?C?DPSEL
      010004B1H   PUBLIC    CODE     NEAR LAB  ?C?ILDXPTR
      010004CDH   PUBLIC    CODE     NEAR LAB  ?C?ISTXPTR
      01000529H   PUBLIC    CODE     NEAR LAB  ?C?LLDXPTR
      0100054BH   PUBLIC    CODE     NEAR LAB  ?C?LSTXPTR
      010004E9H   PUBLIC    CODE     NEAR LAB  ?C?PLDXPTR
      01000508H   PUBLIC    CODE     NEAR LAB  ?C?PSTXPTR
      00000008H   PUBLIC    NUMBER   ---       ?C?XPAGE1RST
      00000096H   PUBLIC    DATA     ---       ?C?XPAGE1SFR
      01000000H   PUBLIC    CODE     NEAR LAB  ?C_STARTUP
      000000E0H   SFRSYM    DATA     BYTE      ACC
      000000F0H   SFRSYM    DATA     BYTE      B
      00000083H   SFRSYM    DATA     BYTE      DPH
      00000082H   SFRSYM    DATA     BYTE      DPL
      00000094H   SFRSYM    DATA     BYTE      MEX1
      00000095H   SFRSYM    DATA     BYTE      MEX2
      00000096H   SFRSYM    DATA     BYTE      MEX3
      00000097H   SFRSYM    DATA     BYTE      MEXSP
      000000A0H   SFRSYM    DATA     BYTE      PPAGE_SFR
      00000081H   SFRSYM    DATA     BYTE      SP
LX51 LINKER/LOCATER V4.06                                                             05/20/2006  16:12:40  PAGE 8


      0100048EH   SYMBOL    CODE     NEAR LAB  ??0001
      010004A6H   SYMBOL    CODE     NEAR LAB  ??0003
      010004BEH   SYMBOL    CODE     NEAR LAB  ??0005
      010004DAH   SYMBOL    CODE     NEAR LAB  ??0007
      010004F6H   SYMBOL    CODE     NEAR LAB  ??0009
      01000515H   SYMBOL    CODE     NEAR LAB  ??000B
      01000536H   SYMBOL    CODE     NEAR LAB  ??000D
      01000558H   SYMBOL    CODE     NEAR LAB  ??000F
      000000F0H   SYMBOL    NUMBER   ---       ?B_MASK
      00000001H   SYMBOL    NUMBER   ---       ?B_VAR_BANKING
      010004ADH   SYMBOL    CODE     NEAR LAB  CSTCODE
      00000000H   SYMBOL    NUMBER   ---       IBPSTACK
      00000100H   SYMBOL    NUMBER   ---       IBPSTACKTOP
      00000080H   SYMBOL    NUMBER   ---       IDATALEN
      010007B8H   SYMBOL    CODE     NEAR LAB  IDATALOOP
      000000B0H   SYMBOL    NUMBER   ---       MEX2VAL
      00000000H   SYMBOL    NUMBER   ---       PBPSTACK
      00010000H   SYMBOL    NUMBER   ---       PBPSTACKTOP
      00000000H   SYMBOL    NUMBER   ---       PDATALEN
      00000000H   SYMBOL    NUMBER   ---       PDATASTART
      00000000H   SYMBOL    NUMBER   ---       PPAGE
      00000000H   SYMBOL    NUMBER   ---       PPAGEENABLE
      010007B5H   SYMBOL    CODE     NEAR LAB  STARTUP1
      00000000H   SYMBOL    NUMBER   ---       XBPSTACK
      00010000H   SYMBOL    NUMBER   ---       XBPSTACKTOP
      00000000H   SYMBOL    NUMBER   ---       XDATALEN
      00000000H   SYMBOL    NUMBER   ---       XDATASTART

      01000000H   BLOCK     CODE     NEAR LAB  LVL=0
      ---         BLOCKEND  ---      ---       LVL=0

      010007B5H   BLOCK     CODE     NEAR LAB  LVL=0
      ---         BLOCKEND  ---      ---       LVL=0

      01000481H   BLOCK     CODE     NEAR LAB  LVL=0
      ---         BLOCKEND  ---      ---       LVL=0

      ---         MODULE    ---      ---       ?C?ISTPTR
      0100056DH   PUBLIC    CODE     ---       ?C?ISTPTR

      ---         MODULE    ---      ---       PRINTF
      0000000AH   PUBLIC    DATA     ---       ?_PRINTF517?BYTE
      0000000AH   PUBLIC    DATA     ---       ?_PRINTF?BYTE
      0000000AH   PUBLIC    DATA     ---       ?_SPRINTF517?BYTE
      0000000AH   PUBLIC    DATA     ---       ?_SPRINTF?BYTE
      01000162H   PUBLIC    CODE     ---       _PRINTF
      01000162H   PUBLIC    CODE     ---       _PRINTF517
      0100015CH   PUBLIC    CODE     ---       _SPRINTF
      0100015CH   PUBLIC    CODE     ---       _SPRINTF517

      ---         MODULE    ---      ---       ?C?STRCPY517
      01000659H   PUBLIC    CODE     ---       ?C?STRCPY517

      ---         MODULE    ---      ---       ?C?CLDPTR
      0100069FH   PUBLIC    CODE     ---       ?C?CLDPTR

      ---         MODULE    ---      ---       ?C?CSTPTR
      010006BDH   PUBLIC    CODE     ---       ?C?CSTPTR

      ---         MODULE    ---      ---       ?C?PLDIIDATA
      010006D4H   PUBLIC    CODE     ---       ?C?PLDIIDATA

      ---         MODULE    ---      ---       ?C?CCASE
      010006E4H   PUBLIC    CODE     ---       ?C?CCASE

LX51 LINKER/LOCATER V4.06                                                             05/20/2006  16:12:40  PAGE 9


      ---         MODULE    ---      ---       PUTCHAR
      0100078EH   PUBLIC    CODE     ---       _PUTCHAR

Program Size: data=36.1 xdata=500 const=0 code=2042
LX51 RUN COMPLETE.  0 WARNING(S),  0 ERROR(S)
